:100000000C945B000C9481000C9481000C94810092
:100010000C9481000C9481000C9481000C9481005C
:100020000C9481000C9481000C9481000C9481004C
:100030000C9481000C9481000C9481000C9481003C
:100040000C947C030C9481000C94CB050C948100DF
:100050000C9481000C9481000C9481000C9481001C
:100060000C9481000C9481007B03000000070002C7
:10007000010000030406000000000000000001026F
:100080000408102040800102040810200102040826
:100090001020040404040404040402020202020204
:1000A0000303030303030000232629000025282B54
:1000B000000024272A0011241FBECFEFD4E0DEBFAA
:1000C000CDBF11E0A0E0B1E0EEE8FEE002C0059097
:1000D0000D92A431B107D9F711E0A4E1B1E001C05C
:1000E0001D92A53BB107E1F710E0CAE6D0E004C0DD
:1000F0002297FE010E944307C836D107C9F70C9426
:10010000A0020C94000061E0809103010E940605AA
:1001100060E0809102010E940605089560E08091F0
:1001200003010E94060561E0809102010E9406051C
:10013000089560E0809103010E94060560E08091CF
:1001400002010E940605089560E0809105010E9469
:10015000060560E0809104010E9406050895209143
:10016000220130912301C9010B978D57934120F44F
:100170003093010120930001089560912201709154
:1001800023016F3F710509F020F4809104010E9462
:100190004B04089560E0809105010E94060560917E
:1001A000220170912301CB0101978F3F910528F423
:1001B000809104010E944B04089561E08091040144
:1001C0000E940605089561E0809105010E940605E0
:1001D0002091220130912301C90101978F3F9105A0
:1001E00048F46FEF70E0621B730B809104010E9472
:1001F0004B04089560E0809104010E940605089573
:100200000F931F93CF93DF93682F8CE291E00E94AE
:10021000BC0260E28CE291E00E94BC02C0E0D0E04F
:1002200002E211E00EC0F801619171918F018CE240
:1002300091E00E94670360E28CE291E00E94BC02C0
:1002400021968091070190910801C817D9075CF3A6
:1002500061E28CE291E00E94D502DF91CF911F9183
:100260000F91089561E0809105010E949F0460E074
:10027000809105010E94060561E0809104010E94C1
:100280009F0460E0809104010E94060561E0809176
:1002900003010E949F0460E0809103010E94060513
:1002A00061E0809102010E949F0460E08091020160
:1002B0000E94060561E08DE00E949F0440E051EE3F
:1002C00060E070E08CE291E00E94AD0208958D3410
:1002D00009F18E343CF4863489F08C34A9F08234F0
:1002E00079F50FC08335C9F084351CF4823541F5AA
:1002F0000EC08435A9F0863519F520C00E94E300B0
:1003000008950E94CA0008950E94830008950E94E3
:100310008E0008950E94990008950E94A4000895F7
:100320002091220130912301C9010B978D579341F0
:1003300038F4309301012093000108950E94BD001C
:100340000895A2C061E08DE00E94060580E490E07F
:1003500090930A01809309018CE291E00E94B60219
:1003600090930A0180930901AA2797FDA095BA2FBF
:1003700020E030E0AC01BD018CE291E00E944C0332
:100380006091090170910A01CB01815490404A9714
:10039000A8F4609306011092080110920701E2E2AE
:1003A000F1E088E090E011921192019797FFFBCF66
:1003B0008FEF9FEF90930801809307016D327105D5
:1003C00031F48FEF9FEF90930C0180930B01CB01E1
:1003D000C0970A97C8F4E0910701F0910801EE0F69
:1003E000FF1FEE5DFE4F808191819C0153E0220F43
:1003F000331F5A95E1F7880F991F820F931F860FBD
:10040000971FC097918380836032710559F54091A1
:100410000701509108018FEF4F3F5807E1F0DCF0E2
:10042000FA01EE0FFF1FEE5DFE4F20910B013091A0
:100430000C0180819181DC012A9FC0012B9F900DCE
:100440003A9F900D11249183808381E090E09093F6
:100450000C0180930B014F5F5F4F50930801409355
:10046000070106C06132710531F06A30710519F07B
:100470006D30710549F460E08DE00E9406058091C1
:1004800006010E94670108958CE291E00E94B20289
:10049000882309F057CF08950E94A1010E94A1036B
:1004A00020911601309117014091180150911901C6
:1004B000261737074807590708F041C00E94A103D3
:1004C0002091000130910101442737FD4095542FC0
:1004D000260F371F481F591F20931601309317010D
:1004E000409318015093190180911A0190911B01BA
:1004F000A0911C01B0911D010196A11DB11D809319
:100500001A0190931B01A0931C01B0931D016DE093
:1005100071E08CE291E00E94C00240911A0150917A
:100520001B0160911C0170911D018CE291E00E9401
:10053000FE0260E171E08CE291E00E94E002089529
:10054000CFEFD4E0DEBFCDBF0E94E8030E943201AE
:100550000E944C02FDCF08950895CB01BA010E947C
:10056000510508950E949205992708950E94A305B8
:1005700008950E94C2050895862F0E9409060895D5
:10058000CB010E9410060895862F0E940906089547
:100590000F931F938C016DE00E94BC026AE0C801BA
:1005A0000E94BC021F910F9108950F931F938C011D
:1005B0000E94BC02C8010E94C8021F910F910895B9
:1005C0000F931F938C010E94C002C8010E94C802B1
:1005D0001F910F9108950F931F938C010E94C402E5
:1005E000C8010E94C8021F910F910895CB01BA0162
:1005F0003327442755270E941D0608952AE00E94AC
:10060000F60208950F931F938C010E94FE02C80109
:100610000E94C8021F910F910895AB0166277727AA
:100620000E94FE0208950F931F938C010E940D03F8
:10063000C8010E94C8021F910F910895EF92FF9286
:100640000F931F93CF93DF93EC017A018B0177FF18
:100650000BC06DE20E94BC0210950095F094E094EE
:10066000E11CF11C011D111D2AE0B801A701CE01FA
:100670000E94F602DF91CF911F910F91FF90EF90B2
:1006800008950F931F938C010E941E03C8010E94BE
:10069000C8021F910F9108952115310521F4642F8F
:1006A0000E94BC0208952A30310519F40E941E03ED
:1006B00008950E94F60208950F931F938C010E94E3
:1006C0004C03C8010E94C8021F910F910895AB010D
:1006D000662757FD6095762F0E941E0308950F939D
:1006E0001F938C010E946703C8010E94C8021F91DA
:1006F0000F910895089508951F920F920FB60F92CB
:1007000011248F939F93AF93BF9380913101909168
:100710003201A0913301B09134010196A11DB11DA8
:100720008093310190933201A0933301B09334014F
:10073000BF91AF919F918F910F900FBE0F901F901F
:10074000189560913101709132018091330190913F
:10075000340127E0660F771F881F991F2A95D1F76C
:100760002DE730E040E050E00E94F006CA01B901F8
:100770000895AF92BF92CF92DF92EF92FF920F93C4
:100780001F935B016C010E94A1037B018C010E94FD
:10079000A1036E197F09800B910B6A157B058C05EF
:1007A0009D05A8F31F910F91FF90EF90DF90CF90E0
:1007B000BF90AF900895019751F0880F991F880F4F
:1007C000991F02972FB7F8940197F1F72FBF08955B
:1007D00078941092310110923201109233011092EC
:1007E000340184B5826084BD84B5816084BD85B5E3
:1007F000826085BD85B5816085BDEEE6F0E08081D3
:1008000081608083E1E8F0E0808182608083808184
:1008100081608083E0E8F0E0808181608083E1EBAB
:10082000F0E0808184608083E0EBF0E08081816093
:100830008083EAE7F0E08081846080838081826049
:100840008083808181608083808180688083109232
:10085000C10008958093130108959091130192951A
:10086000990F990F907C8F70982B90937C008091BA
:100870007A00806480937A0080917A0086FDFCCFB4
:1008800020917800809179009927982F8827332725
:10089000822B932B08951F93CF93DF93182FEB0197
:1008A00061E00E949F04E12FFF27E659FF4F8491EA
:1008B000833051F480918000806880938000D093D1
:1008C0008900C093880037C0843051F48091800043
:1008D000806280938000D0938B00C0938A002BC0ED
:1008E000813029F484B5806884BDC7BD24C08230BE
:1008F00029F484B5806284BDC8BD1DC0863041F432
:100900008091B00080688093B000C093B30013C0A2
:10091000873041F48091B00080628093B000C09332
:10092000B40009C0C038D10514F460E001C061E032
:10093000812F0E940605DF91CF911F910895282FE6
:100940003327C90182589F4FFC0194912E563F4F87
:10095000F9018491882381F0E82FFF27E055FF4FAC
:10096000E491FF27662329F4808190958923808371
:1009700008958081892B80830895482F5527CA01C7
:1009800086599F4FFC012491CA0182589F4FFC0158
:1009900094914E565F4FFA0134913323A1F12223F3
:1009A00031F1233021F4809180008F7705C024300D
:1009B00031F4809180008F7D8093800018C02130B9
:1009C00019F484B58F7704C0223021F484B58F7D6B
:1009D00084BD0DC0263021F48091B0008F7705C012
:1009E000273029F48091B0008F7D8093B000E32FF1
:1009F000FF27EA55FF4FE491FF278081892319F0F3
:100A000081E090E0089580E090E00895482F552718
:100A1000CA0186599F4FFC012491CA0182589F4FF9
:100A2000FC0194914E565F4FFA0134913323C1F18A
:100A3000222331F1233021F4809180008F7705C08B
:100A4000243031F4809180008F7D8093800018C025
:100A5000213019F484B58F7704C0223021F484B595
:100A60008F7D84BD0DC0263021F48091B0008F773A
:100A700005C0273029F48091B0008F7D8093B000AD
:100A8000E32FFF27E555FF4FE491FF27662329F465
:100A9000808190958923808308958081892B80832C
:100AA0000895EF92FF920F931F937B018C0122E038
:100AB00030E040E050E00E941207205C3D4B404F88
:100AC0005F4FCA01B901A80197010E941207215086
:100AD000304040405040BB2757FDBA95A52F942F7A
:100AE000832F2F5F3F4F4F4F5F4F8093C5002150A3
:100AF0002093C400E1ECF0E08081806180838081FC
:100B0000886080838081806880831F910F91FF902F
:100B1000EF900895982F8091C00085FFFCCF9093AF
:100B2000C600089580912F019091300120912D01F0
:100B300030912E01821B930B80589F4F60E870E02C
:100B40000E94DD06089540912D0150912E01809163
:100B50002F01909130018417950719F48FEF9FEFC3
:100B60000895FA01EB5CFE4F2081CA01019660E80E
:100B700070E00E94DD0690932E0180932D01822F5C
:100B80009927089580912D0190912E019093300125
:100B900080932F0108951F920F920FB60F92112488
:100BA0002F933F934F935F936F937F938F939F9375
:100BB000AF93BF93EF93FF934091C600E0912F0155
:100BC000F0913001CF01019660E870E00E94DD06EF
:100BD0009C0180912D0190912E012817390739F041
:100BE000EB5CFE4F40833093300120932F01FF9147
:100BF000EF91BF91AF919F918F917F916F915F9195
:100C00004F913F912F910F900FBE0F901F9018950D
:100C100008950E948A0508958AE00E9409060895B1
:100C2000CF93DF93EC0103C021960E9409068881CF
:100C30008823D1F7DF91CF9108952F923F924F9261
:100C40005F926F927F928F929F92AF92BF92CF925C
:100C5000DF92EF92FF920F931F93CF93DF93CDB765
:100C6000DEB7A0970FB6F894DEBF0FBECDBF6B0105
:100C70007C0119012A01611571058105910521F495
:100C800080E30E9409064BC06624772443015E017D
:100C90000894A11CB11C8501060D171DC701B601E2
:100CA000A20191010E94F006F80160830894611C82
:100CB000711C811C911CC701B601A20191010E9407
:100CC000F00669017A01211531054105510519F731
:100CD00073010894E108F108EA0CFB1CAA24BB2468
:100CE000650111C0F70180818A3010F4805D01C078
:100CF000895C0E9409060894A108B108C108D108BE
:100D00000894E108F10888279927DC0186199709DA
:100D1000A809B909A816B906CA06DB0619F7A096EC
:100D20000FB6F894DEBF0FBECDBFDF91CF911F91FC
:100D30000F91FF90EF90DF90CF90BF90AF909F907A
:100D40008F907F906F905F904F903F902F9008957D
:100D5000EF92FF920F931F937B018C0197FF0BC0C3
:100D60008DE20E94090610950095F094E094E11C34
:100D7000F11C011D111D2AE030E040E050E0C801E7
:100D8000B7010E941D061F910F91FF90EF900895EB
:100D900020E130E040E050E00E941D06089528E088
:100DA00030E040E050E00E941D06089522E030E06F
:100DB00040E050E00E941D06089597FB092E07268B
:100DC0000AD077FD04D049D006D000201AF47095DF
:100DD00061957F4F0895F6F7909581959F4F0895FF
:100DE000A1E21A2EAA1BBB1BFD010DC0AA1FBB1F2F
:100DF000EE1FFF1FA217B307E407F50720F0A21BA1
:100E0000B30BE40BF50B661F771F881F991F1A940D
:100E100069F760957095809590959B01AC01BD0137
:100E2000CF01089597FB092E05260ED057FD04D05B
:100E3000D7DF0AD0001C38F45095409530952195A5
:100E40003F4F4F4F5F4F0895F6F7909580957095FF
:100E500061957F4F8F4F9F4F0895AA1BBB1B51E198
:100E600007C0AA1FBB1FA617B70710F0A61BB70B1A
:100E7000881F991F5A95A9F780959095BC01CD01BF
:0E0E80000895EE0FFF1F0590F491E02D0994E8
:100E8E00E8030B0A090840FFFFFFFF010056200090
:040E9E00202100010E
:00000001FF
